:100000000C9462000C948A000C948A000C948A0070
:100010000C948A000C948A000C948A000C948A0038
:100020000C948A000C948A000C948A000C948A0028
:100030000C948A000C948A000C948A000C948A0018
:100040000C944D040C948A000C9474050C948A0052
:100050000C948A000C948A000C948A000C948A00F8
:100060000C948A000C948A000000000024002700F1
:100070002A0000000000250028002B0000000000DE
:1000800023002600290004040404040404040202DA
:100090000202020203030303030301020408102007
:1000A0004080010204081020010204081020000012
:1000B0000007000201000003040600000000000029
:1000C0000000050711241FBECFEFD8E0DEBFCDBF73
:1000D00011E0A0E0B1E0E4EFF1E102C005900D9283
:1000E000A836B107D9F712E0A8E6B1E001C01D9229
:1000F000A334B107E1F710E0C4ECD0E004C02297CC
:10010000FE010E94F408C23CD107C9F70E944604D0
:100110000C94F8080C940000CF92DF92FF920F939A
:100120001F93CF93DF93F82E062F142F862F61E0B5
:100130000E9407058F2D61E00E9407058F2D60E06A
:100140000E942705802F60E00E942705C7E0D0E0CD
:10015000C12EDD24802F60E00E942705B6010C2E01
:1001600002C0759567950A94E2F761708F2D0E9421
:100170002705802F61E00E9427058F2D60E00E94F7
:10018000270521978FEFCF3FD80721F7802F60E019
:100190000E942705DF91CF911F910F91FF90DF9073
:1001A000CF900895CF92DF92EF92FF920F931F931B
:1001B000CF93DF936C01C0E0D0E07B010027F7FC18
:1001C0000095102F79C08091540160E00E942705AE
:1001D0006091560170915701809158019091590199
:1001E00040916D010E948C00609156017091570101
:1001F0008091580190915901409177010E948C00A3
:100200006091560170915701809158019091590168
:10021000409181010E948C006091560170915701BC
:10022000809158019091590140918B010E948C005E
:100230008091540161E00E942705C801B7010E9426
:10024000A3048091540160E00E942705609156014B
:1002500070915701809158019091590140E00E949E
:100260008C006091560170915701809158019091D6
:10027000590140E00E948C00609156017091570135
:10028000809158019091590140E00E948C0060914A
:10029000560170915701809158019091590140E0A9
:1002A0000E948C008091540161E00E942705C801E2
:1002B000B7010E94A3042196CC15DD050CF483CF71
:1002C000DF91CF911F910F91FF90EF90DF90CF9032
:1002D0000895CF92DF92EF92FF920F931F93CF93E7
:1002E000DF936C01C0E0D0E07B010027F7FC0095B4
:1002F000102F75C08091540160E00E942705609125
:1003000056017091570180915801909159014FEF1A
:100310000E948C00609156017091570180915801A4
:10032000909159014FEF0E948C006091560170919D
:10033000570180915801909159014FEF0E948C0014
:100340006091560170915701809158019091590127
:100350004FEF0E948C008091540161E00E942705BC
:10036000C801B7010E94A3048091540160E00E947B
:100370002705609156017091570180915801909125
:10038000590140E00E948C00609156017091570124
:10039000809158019091590140E00E948C00609139
:1003A000560170915701809158019091590140E098
:1003B0000E948C0060915601709157018091580104
:1003C0009091590140E00E948C008091540161E0BD
:1003D0000E942705C801B7010E94A3042196CC15ED
:1003E000DD050CF487CFDF91CF911F910F91FF9026
:1003F000EF90DF90CF900895EF92FF920F931F93AD
:10040000E0905A01F0905B0100915C0110915D0158
:100410008091540160E00E9427052091560130919F
:100420005701C8016AE070E00E948E08FB01E359A1
:10043000FE4F8091580190915901B90140810E946D
:100440008C0080915A0190915B0162E070E00E9403
:100450008E089C012B563E4FC8016AE070E00E9456
:100460008E08FC01E958FE4FD9014C918081482B40
:1004700040936C0160915601709157018091580131
:10048000909159010E948C002091560130915701A2
:10049000C7016AE070E00E948E08FB01EF57FE4F33
:1004A0008091580190915901B90140810E948C00BE
:1004B0002091560130915701C7016AE070E00E9417
:1004C0008E08FC01E557FE4F80915801909159012B
:1004D000B90140810E948C008091540161E00E942A
:1004E00027051F910F91FF90EF9008958F929F9293
:1004F000AF92BF92CF92DF92EF92FF920F931F9332
:10050000CF93DF9380E392E00E94AA06882309F448
:10051000C4C080E392E00E94BE068336910509F0D4
:10052000B8C010926B0110926A0180E392E060E023
:1005300071E00E949507C6E0D0E035E0832E912C53
:1005400024E0A22EB12C93E0C92ED12C82E0E82E1B
:10055000F12C01E010E096C080E392E00E94AA0630
:10056000882309F48FC080E392E00E94BE069C01BC
:100570008C36910581F480916A0190916B01892BF1
:1005800009F041C010936B0100936A0180E392E08F
:100590006CE071E011C08F36910589F480916A0199
:1005A00090916B01019779F5F0926B01E0926A01ED
:1005B00080E392E068E171E00E94950763C08336B2
:1005C000910579F480916A0190916B010297D9F4B9
:1005D000D0926B01C0926A0180E392E060E071E02A
:1005E000EBCF8B36910579F480916A0190916B0184
:1005F000039749F4B0926B01A0926A0180E392E004
:1006000064E271E0D9CF80916A0190916B018430EE
:100610009105B9F430935D0120935C0190926B01D8
:1006200080926A0180E392E060E371E00E947607C5
:1006300060915C0170915D0180E392E00E945F082F
:1006400021C00597D9F430935B0120935A01D093D0
:100650006B01C0936A0180E392E062E471E00E9462
:10066000760760915A0170915B0180E392E00E94ED
:100670005F08109269011092680104C0D0936B0169
:10068000C0936A0180916A0190916B0106970CF406
:1006900063CF80E392E00E94E6060E9495042091D9
:1006A0009F013091A0014091A1015091A201621BD4
:1006B000730B840B950B685E734080409040D8F0BC
:1006C0008091680190916901892BA9F40E94950499
:1006D00060939F017093A0018093A1019093A20168
:1006E0000E94FC0180915A0190915B0101979093C7
:1006F0005B0180935A0180915A0190915B0197FFB1
:100700000FC080915C0190915D01019790935D0114
:1007100080935C018BE390E090935B0180935A019E
:1007200080915C0190915D0197FF10C081E090E0A5
:10073000909369018093680110925D0110925C01B1
:1007400085E090E068EE73E00E94D200DF91CF91E7
:100750001F910F91FF90EF90DF90CF90BF90AF90DF
:100760009F908F9008958091540161E00E94070549
:1007700080E392E040E051EE60E070E00E94B1055D
:100780008FE680936D0183E080936E01FDE5F09329
:100790006F0187E58093700183E38093710186E7A1
:1007A000809372018EE78093730183E480937401D8
:1007B000EFE7E093750177E770937601109295016A
:1007C00081E0809396011092970180939801109296
:1007D000990180939A0110929B0180939C01109241
:1007E0009D0180939E018EED8093770186E080933A
:1007F00078018AEB809379018EEA80937A0196E6FC
:1008000090937B018CEE80937C018CEF80937D0133
:1008100086E880937E018EEF80937F018EEE809339
:1008200080016BE76093810150E650938201F09361
:10083000830145E7409384019093850137E330932A
:1008400086012FE32093870181E680938801E0935E
:10085000890170938A0160938B0150938C01F0930E
:100860008D0140938E0190938F01309390012093DE
:10087000910180939201E09393017093940182E03F
:1008800090E064EF71E00E94690108950E94CD0438
:100890000E94B3030E947602FDCF1F920F920FB603
:1008A0000F9211242F933F938F939F93AF93BF93F6
:1008B0008091A7019091A801A091A901B091AA01EE
:1008C0003091AB010196A11DB11D232F2D5F2D3756
:1008D00020F02D570196A11DB11D2093AB018093EF
:1008E000A7019093A801A093A901B093AA018091B8
:1008F000A3019091A401A091A501B091A601019638
:10090000A11DB11D8093A3019093A401A093A50103
:10091000B093A601BF91AF919F918F913F912F917D
:100920000F900FBE0F901F9018958FB7F8942091DD
:10093000A7013091A8014091A9015091AA018FBF50
:10094000B901CA010895EF92FF920F931F937B01A3
:100950008C018FB7F8944091A7015091A801609144
:10096000A9017091AA018FBF2FB7F8948091A701B8
:100970009091A801A091A901B091AA012FBF841B59
:10098000950BA60BB70BE816F9060A071B0760F7CD
:100990001F910F91FF90EF900895789484B5826035
:1009A00084BD84B5816084BD85B5826085BD85B513
:1009B000816085BDEEE6F0E0808181608083E1E8C2
:1009C000F0E0808182608083808181608083E0E8C4
:1009D000F0E0808181608083E1EBF0E080818460E1
:1009E0008083E0EBF0E0808181608083EAE7F0E0E3
:1009F0008081846080838081826080838081816047
:100A000080838081806880831092C1000895282FA0
:100A100030E0C90186569F4FFC0194912A573F4F01
:100A2000F9018491882391F0E82FF0E0EE0FFF1F89
:100A3000E859FF4FA591B491662329F48C919095C4
:100A400089238C9308958C91892B8C930895482F3A
:100A500050E0CA0182559F4FFC012491CA0186567D
:100A60009F4FFC0194914A575F4FFA013491332311
:100A7000D1F1222331F1233021F4809180008F774E
:100A800005C0243031F4809180008F7D80938000F8
:100A900018C0213019F484B58F7704C0223021F4B6
:100AA00084B58F7D84BD0DC0263021F48091B000C7
:100AB0008F7705C0273029F48091B0008F7D809317
:100AC000B000E32FF0E0EE0FFF1FEE58FF4FA591AF
:100AD000B491662329F48C91909589238C93089581
:100AE0008C91892B8C9308951F920F920FB60F92C1
:100AF00011242F933F934F935F936F937F938F9323
:100B00009F93AF93BF93EF93FF934091C600E09103
:100B10002C02F0912D02CF01019660E870E00E9456
:100B20008E089C0180912E0290912F022817390780
:100B300039F0E455FE4F408330932D0220932C0270
:100B4000FF91EF91BF91AF919F918F917F916F91A5
:100B50005F914F913F912F910F900FBE0F901F907B
:100B600018955F926F927F928F929F92AF92BF92F1
:100B7000CF92DF92EF92FF920F931F93CF93DF9369
:100B8000EC013A014B01413482E458078FE06807D9
:100B900080E078070CF07FC060E874E88EE190E0B8
:100BA000A40193010E94C3082150304040405040AE
:100BB000CA01B90122E030E040E050E00E94C308E1
:100BC00059016A01A60195012095309540955095EF
:100BD00094E0220F331F441F551F9A95D1F760E010
:100BE00074E284EF90E00E94C308CA01B9012FEFBC
:100BF00030E040E050E00E946F08A40193010E94A1
:100C0000C308C90181509F4F181619061CF4522EB3
:100C10005A9403C055245394521A60E079E08DE34E
:100C200090E0A40193010E94C3082150304040404D
:100C30005040CA01B90122E030E040E050E00E949B
:100C4000C308209530954095509583E0220F331FBF
:100C5000441F551F8A95D1F760E074E284EF90E05D
:100C60000E94C308CA01B9012FEF30E040E050E014
:100C70000E946F08A40193010E94C308C90181501A
:100C80009F4F181619061CF4822F815002C081E074
:100C9000821B851500F5E885F98581E090E00A88DA
:100CA00002C0880F991F0A94E2F7808360E079E020
:100CB0008DE390E0A40193010E94C30821503040CD
:100CC00040405040CA01B90122E030E040E050E02D
:100CD0000E94C30804C0E885F98510829501EC8163
:100CE000FD813083EE81FF812083EA85FB852081B1
:100CF00041E050E0CA010E8402C0880F991F0A9497
:100D0000E2F7282B2083EA85FB852081CA010F8426
:100D100002C0880F991F0A94E2F7282B2083EA85E6
:100D2000FB858081088802C0440F551F0A94E2F7B2
:100D3000842B8083DF91CF911F910F91FF90EF90D3
:100D4000DF90CF90BF90AF909F908F907F906F90EB
:100D50005F900895DC011296ED91FC911397E05895
:100D6000FF4F8191919180589F4F20813181821B4B
:100D7000930B60E870E00E948E080895CF93DF9394
:100D8000DC011296ED91FC911397EF01CE57DF4FE6
:100D900048815981E058FF4F80819181E058F040AF
:100DA0008417950719F42FEF3FEF0CC0E40FF51FE0
:100DB0002081CA01019660E870E00E948E08998344
:100DC000888330E0C901DF91CF910895DC0112964C
:100DD000ED91FC911397EE57FF4F80819181929393
:100DE00082930895FC01A085B18521898C9190E0C2
:100DF000022E02C0959587950A94E2F780FFF6CF00
:100E00000484F585E02D6083089582E691E0909357
:100E10003102809330028CEA91E090933302809308
:100E2000320285EC90E0909335028093340284EC9A
:100E300090E0909337028093360280EC90E090939C
:100E400039028093380281EC90E090933B028093CA
:100E50003A0286EC90E090933D0280933C0284E05D
:100E600080933E0283E080933F0287E080934002BC
:100E700085E08093410281E08093420208950F93C0
:100E80001F93CF93DF938C01EB0109C02196D8010A
:100E9000ED91FC910190F081E02DC80109956881E8
:100EA0006623A1F7DF91CF911F910F910895EF92E3
:100EB000FF920F931F93CF93DF938C017B01EA0185
:100EC0000CC0D7016D917D01D801ED91FC9101908D
:100ED000F081E02DC80109952197209791F7DF91C6
:100EE000CF911F910F91FF90EF900895DC01ED914C
:100EF000FC910280F381E02D099508950F931F93D3
:100F00008C01DC01ED91FC910190F081E02D6DE010
:100F10000995D801ED91FC910190F081E02DC80177
:100F20006AE009951F910F9108950F931F938C010B
:100F30000E947607C8010E947E071F910F910895B5
:100F40002F923F924F925F926F927F928F929F92D9
:100F5000AF92BF92CF92DF92EF92FF920F931F93C7
:100F6000DF93CF93CDB7DEB7A0970FB6F894DEBF6F
:100F70000FBECDBF1C016A017B0141155105610502
:100F8000710549F4DC01ED91FC910190F081E02DB7
:100F900060E3099554C0882499245401422E5524B5
:100FA0006624772401E010E00C0F1D1F080D191DA9
:100FB000C701B601A30192010E94A108F801608354
:100FC0000894811C911CA11CB11CC701B601A3018E
:100FD00092010E94A108C901DA016C017D01C114CE
:100FE000D104E104F104F1F681E0E82EF12CEC0EDD
:100FF000FD1EE80CF91C3E010894611C711CD50112
:10100000C4010197A109B1096C01C818D90814C01D
:10101000F601EE0DFF1D60816A3010F4605D01C0C5
:10102000695CD101ED91FC910190F081E02DC1014D
:1010300009950894E108F1086E147F0449F7A09619
:101040000FB6F894DEBF0FBECDBFCF91DF911F91D9
:101050000F91FF90EF90DF90CF90BF90AF909F9057
:101060008F907F906F905F904F903F902F9008955A
:10107000EF92FF920F931F93CF93DF93EC017A01CE
:101080008B0177FF0FC0E881F9810190F081E02D9D
:101090006DE2099510950095F094E094E11CF11C27
:1010A000011D111DCE01B801A7012AE00E94A00771
:1010B000DF91CF911F910F91FF90EF9008950F93C3
:1010C0001F938C01AB01662757FD6095762F0E9418
:1010D0003808C8010E947E071F910F910895629FF2
:1010E000D001739FF001829FE00DF11D649FE00D20
:1010F000F11D929FF00D839FF00D749FF00D659F81
:10110000F00D9927729FB00DE11DF91F639FB00D7F
:10111000E11DF91FBD01CF011124089597FB092E90
:1011200007260AD077FD04D049D006D000201AF453
:10113000709561957F4F0895F6F7909581959F4F33
:101140000895A1E21A2EAA1BBB1BFD010DC0AA1F08
:10115000BB1FEE1FFF1FA217B307E407F50720F020
:10116000A21BB30BE40BF50B661F771F881F991F9B
:101170001A9469F760957095809590959B01AC01E4
:10118000BD01CF01089597FB092E05260ED057FD0E
:1011900004D0D7DF0AD0001C38F450954095309524
:1011A00021953F4F4F4F5F4F0895F6F790958095EB
:1011B000709561957F4F8F4F9F4F0895AA1BBB1B62
:1011C00051E107C0AA1FBB1FA617B70710F0A61B47
:1011D000B70B881F991F5A95A9F780959095BC0168
:1011E000CD010895EE0FFF1F0590F491E02D0994B5
:0411F000F894FFCFA1
:1011F4006465746563746164612063006465746527
:101204006374616461206C00646574656374616413
:1012140061206F00646574656374616461206B00B0
:1012240064657465637461646F206D696E7574655B
:10123400200064657465637461646F207365636F13
:101244006E64200008000C000B003B000E00000040
:081254000000F2063F075707F6
:00000001FF
